:020000040000FA
:0E0000000219FDD2D3A68A08C2D33202119192
:0300130002054E95
:0F001B00302F0AD2D3B284868B08C2D33281D75A
:10002B0075C800203E0653E6DF020436752741856E
:09003B0055CC8556CD43E6203278
:03005B0002055C3F
:10006300302454C521C59B30E61620181002043BEA
:1000730053917FC050C05122759B808136C5213278
:10008300C52120180132759100856C94856D957595
:1000930050FE202410C56EF552047553FE6003759F
:1000A300500014C56E75910443E680C21832203E99
:1000B30004D0E0012B8045759B80C0E0E59B65275C
:1000C30020E63120182B103821C2CA10CFE0E5CC2E
:1000D300F4F5CCE5CDF4F5CD303E0FC0D0C3E5CC7F
:1000E3009555E5CD95564012D0D0B23ED2CAD0E058
:1000F30032D0E032D0E020188D32D0D08555CC8577
:1001030056CD80E6D0E075C80053E6DF813604069D
:10011300080C10182030406080A0C00000000000D0
:1001230000000000000000000000000000000000CC
:1001330000000000000000000000000000000000BC
:1001430000000000000000000000000000000000AC
:10015300000000000000000000000000000000009C
:10016300000000000000000000000000000000008C
:10017300000000000000000000000000000000007C
:10018300000000000000000000000000000000006C
:10019300000000000000000000000000000000005C
:1001A300000000000000000000000000000000004C
:1001B300000000000000000000000000000000003C
:1001C300000000000000000000000000000000002C
:1001D300000000000000000000000000000000001C
:1001E300000000000000000000000000000000000C
:1001F30000000000000000000000000000C55204E1
:1002030004700714C5528553503214C55232D2A01C
:10021300C2AFC294D29575D536D2AF759F32754FA2
:10022300266169D2A0C2AF75D52DD2AF759F037574
:100233004F376169D2A0C2AFC295D29375D52DD283
:10024300AF759F31754F4C6169D2A0C2AF75D51B95
:10025300D2AF759F23754F5D6169D2A0C2AFC293C0
:10026300D29475D51BD2AF759F30754F726169D229
:10027300A0C2AF75D536D2AF759F13754F11D21A81
:100283006169D2A0C2AFC295D29475D536D2AF758B
:100293009F31754F9A6169D2A0C2AF75D51BD2AF9A
:1002A300759F03754FAB6169D2A0C2AFC294D2935D
:1002B30075D51BD2AF759F32754FC06169D2A0C28D
:1002C300AF75D52DD2AF759F13754FD16169D2A08C
:1002D300C2AFC293D29575D52DD2AF759F30754FEE
:1002E300E66169D2A0C2AF75D536D2AF759F2375CB
:1002F3004F85D21A61693024068045D2198136753B
:100303009100856994856A957550FE202410C56B0C
:10031300F552047553FE600375500014C56B759157
:100323000443E680C219C218202002D2187527415F
:10033300759BB075C8008555CC8556CD43E62032F4
:10034300C2AF759100856994856A95759104D2AFA2
:100353007550FE43E680C219D21875218075274176
:1003630043E620020063302426C0D0C2AF7591005B
:10037300C5942563C594C5953564C595759104D217
:10038300AF5003439180D0D07550F943E680327566
:1003930091008563948564957550F9202410C56593
:1003A300F552047553F9600375500014C5657591D2
:1003B3000443E6803253E6DF75C800C2A07591009E
:1003C300856694856795854F50202410C568F5523E
:1003D30004854F53600375500014C5687591044339
:1003E300E680C0E0C0D0E55C64036038D21BE8C59A
:1003F30057F8C3E5F9A660F56096F608E5FAA66135
:10040300F56120DF0D96F608E54DA662F56296F6D6
:10041300807420E7F096F608E54D0480ED20E7119F
:100423000562806C85F960E5FAF561854D6220DF30
:10043300EC805D20240761B8C521759B80C2AF7530
:100443009100856694856795759104D2AF854F5069
:1004530043E68053E6DF75C800C2A0C0E0C0D0E524
:100463005C640360BFD21BE8C557F8C3E5F9A66017
:10047300F56096F608854D62E5FA20DF20A661F562
:100483006196F6087600E8040444F0C557F8055C65
:10049300E5245403600E2021020532801D20E7DD90
:1004A300056280D9A218922730190F20230C201837
:1004B30009B193D226D0D0D0E032C3E55B95354065
:1004C30009C290C291C29275D53FD0D0D0E053E615
:1004D300DFC21932C2A8C0D0C0E0C28ED22D758A45
:1004E30000E508B4B72E30332DD22FD28443A410A5
:1004F3007508B9758921538EF0758BCE85748C85FB
:10050300738AC28DC28FD2BBD28CD28E43A80AD03B
:10051300E0D0D032D22E85718B7508A7D2A8D2AA8B
:10052300D0E0D0D032E54E240CF54EE52260021522
:1005330022C3E5396005753A00A149E53A2401F57E
:100543003A5003753AFFD0D0D0E032C2AA85718BFE
:10055300D28E85F94A85FA4B32C0E0E5F730E619C9
:1005630053F7DFE5F9E5FA30E10F853BFB853CFC0A
:10057300853DE9853EEA53F7BF10DF03D0E032C281
:10058300DF054DC0D0E54E954D609AD0D0D0E03216
:10059300C2AF75910075C800759B00D2AFC2AFC2E0
:1005A30090C291C292C293C294C29575D53FD2AF05
:1005B300227901801879038014790A8010790F80D9
:1005C3000C791E80087964800479C88000781474DB
:1005D300F0000000D5E0FAD8F6D9F22279018014B0
:1005E30079038010790A800C791E8008796480046D
:1005F30079C8800075910075944C7595A075910428
:1006030053E67FE9C0E0F1DBD0E0F9E59130E7F3B1
:10061300D9E22278FF20202879A1E76023E55960F9
:100623001F74C48559F0848536F030210375F005B5
:10063300A4F8C5F0600278FFC3E895425002A842CF
:10064300884122C3E55D94E4E55E9400E5415003EF
:10065300148001046002F541220543C3E543940875
:10066300404F30EDF475430079A0E76043E5BE7079
:1006730006E5446019800DC3E5BD9544600EE5446D
:100683005005600A1480070460FA8002E544F544CB
:10069300C39548401B7540C0C39404401375408004
:1006A300C39404400B754040C39404400375400059
:1006B30022E5402410500274FFF54022743279A6DB
:1006C30087F0A4C5F0A2F733F54222755D00755E8D
:1006D300F0227A1C7B3C80127A147B4B800C7A10BC
:1006E3007B5A80067A0A7B788000EFD5E001227975
:1006F30002E4C294D5E0FDD291D5E0FDC291D5E0EC
:10070300FDD294D5E0FDE920E002D29030E002D2A0
:1007130092EFD5E0FDE920E002C29030E002C29200
:100723007496D5E0FDD9CAEAF8D5E0FDD8FBDBBA6B
:10073300C294227886760908760178927603087641
:1007430028087650087604087602087607087601AA
:10075300087600087600227888E6C39403D23250E4
:1007630002C232C230E630E102D230A23092317896
:1007730086E6149001119378A6F67886E6F536C3DB
:1007830094025003753602789CE67535FFB4020374
:100793007535A0B4030375358278A0E6F860067456
:1007A300282409D8FCF5482278A5E6F95403C28524
:1007B3007002D285E9540CC2867002D286E95430A5
:1007C300C2877002D287E954C0C2B37002D2B32287
:1007D300120B9C221211C422102DF5A22BB033B0A0
:1007E3002F40F122754600754700B19375801F7540
:1007F300F1F075A4E075801F75D4FF7590C075F294
:100803003F75A53F7590C075D53F75A00075A601CE
:10081300E5B525E0600975A71075CF0075A70075CC
:10082300E34075E2021205931207361213CC754C9E
:10083300017557F07558F0755102C2AF1205CC78A7
:100843009886071206D51205C01205C01205C012FC
:1008530006DB1205C01205C01205C01206E112051F
:10086300C01205C01205C01206E71206E71205C83A
:100873001207AB22C2AF53A4EFD28475460075476B
:1008830000AAE475E4C478FA79FA308409D9FBD86C
:10089300F7021C008AE422C2AF12075A120593C260
:1008A3002575D84075D90975F781759E037596022C
:1008B30075DA4275DB4275A82175E61043B80175F8
:1008C3009B80759D3075D10C75BC5975BB1075E84F
:1008D3008075B2017534001205B42230580675E4F0
:1008E3004CD22B2275E4C4C22B22C2AF7898860760
:1008F300A22B40071206E71206E7221206E11206B0
:10090300E122D2AF1205F31205EFC3E5399401409A
:100913000280EFC2AFA22B78988607402CC0071243
:1009230006D5D2AF1205EFC2AFD0071206D5C00766
:10093300D2AF1205EFC2AFD0071206D5C007D2AFB0
:100943001205EFC2AFD00780091206E71206E712BD
:1009530006E7C289D2AF1205F322E4F55DF55EF531
:100963005FF530F531752000052030014575200015
:100973000530E530F4703B0531789AE67819146058
:1009830012783214600D787D14600878FA146003CD
:10099300753100C3E5319840191205931205B4155A
:1009A3003175300078998607C2AF1206E7D2AF12CD
:1009B30005EF1205E7E5227002C3221205DF302896
:1009C300A7C3E5399401500AC3E56F9401501E0291
:1009D300096B1205EFE5227002C322756F00757073
:1009E30000D3227546A57547F112140622AF6F1284
:1009F300149F754600754700C22880BFC2AF755764
:100A0300F07558F0755C00D2AF120593E4F543F529
:100A130023F524F55B7543081205DF75E89030ED87
:100A2300FDA8BDE5BE7001F8884412065C75430855
:100A33001206BF854240854241303207C230302919
:100A430002D230D220753200E4C2AF85F96085FA54
:100A530061854D62D2AFF55DF55E755F04755950E2
:100A6300120FF012116220300812029A12028580CE
:100A73000612022612021175E890E55CC394045035
:100A830016102618101B17102D23A22BB033B02FCE
:100A93004016101A1D80E312059380FE616AD1236C
:100AA300120FF012116280D21211C480CD120B9C6E
:100AB30080C82024031206163024031206461206A9
:100AC3005C30202785424079187A0CC3E53299407F
:100AD3000EC220D2218A33854240854241800CC315
:100AE300E53994014003020A7A617230211F202301
:100AF3001CE533147006C221D222417AF533203229
:100B030007C3E53994014003020A7A806275340011
:100B130020320F78FA79A4E760027803C3E53A98A4
:100B2300504DE522604930321520300520290780D9
:100B33000D3029028008202305D22385424078F016
:100B43003023058542407819C3E559985003020ABA
:100B53007A30231BC223C230302902D230D221750E
:100B63003312854240417A0534E539600261757577
:100B73003400120593752400C2891205EF12059300
:100B830075230078A4E66006D293D294D295C3E588
:100B93003494044002C322D322102E0CE4AE72FC20
:100BA300FBFA790878A78002A15CE6FDC39CC39E8B
:100BB30040F69EEB33FB08E6FCC39DC39E40E99ED3
:100BC300EB33FB08E6FDC39CC39E40DC9EEB33FB8B
:100BD30008E6FCC39DC39E40CF9EEB33FB08E6FDB6
:100BE300C39CC39E40C29EEB33FB08E6FCC39DC37C
:100BF3009E40B59EEB33FB08E6FDC39CC39E40A815
:100C03009EEB33FB08E6FCC39DC39E409B9EEB33E8
:100C1300FB088002A15CE6FDC39CC39E40F69EEAEE
:100C230033FA08E6FCC39DC39E40E99EEA33FA0803
:100C3300E6FDC39CC39E40DC9EEA33FA08E6FCC390
:100C43009DC39E40CF9EEA33FA08E6FDC39CC39E34
:100C530040C29EEA33FA08E6FCC39DC39E40B59E9C
:100C6300EA33FA08E6FDC39CC39E40A89EEA33FA22
:100C730008E6FCC39DC39E409B9EEA33FA08EBC47F
:100C83006B6A54F0F9EAC4302B01F454F0C3996051
:100C930002A15CEBF4C454F0F9EAF4C4540F49FA2A
:100CA300EBF4C4540FFBC3EAF99460FAEB9400FB32
:100CB3005020C3E97B007A0079006016C313500605
:100CC300F9C3956F600AE9F56F75700079008002CA
:100CD3000570303227C3EA94D0F8EB9407F9400B40
:100CE300E8FAE9FB202909D2298005302902C22923
:100CF300203102B229C3EA33FAEB33FBEB2B3B3B44
:100D0300F9C3EB13FBEA13FAEA29FAEB3400FB30DD
:100D1300E3047AFF7BFFE5245403601B202218E5DC
:100D23004233F9EB7007C3E99A4002E9FAE534C4A8
:100D3300332AFAEB3400FBC3EA33C4540FF8EB3322
:100D4300C454F048F87005EA60027801E57960025E
:100D53001579802475220A80140579E579700215C6
:100D630079C3E5799432500280EA753900202F0760
:100D7300D2AAD2A87508A7228839D228E8600375B9
:100D83003A00C3E540FC95414002AC41C3EC9539C0
:100D93005008EC75F008A4FAABF0EBF4131392D5FA
:100DA300A2E75401F9EAF4FC13A2D513F8E54C23A6
:100DB300F54CEC5403243783554C600BE82401E9CC
:100DC300340020E10208F9C3E89407FAE99400FB30
:100DD30050047A007B00883B893C8A3D8B3E752218
:100DE3000A53F7DF43F740202F0343E610A17000B7
:100DF300115577C3EC13FCEB13FBEA13FA860508D2
:100E0300860608860708084300F08858C3EF940C49
:100E130040027F0CC3ED33FDEE33FEEF33FFE10CF5
:100E2300A858302477AA5DAB5EC3EAC4540FFCEB29
:100E3300C4FD54F04CCA9AFAED540FCB9BFBE60366
:100E430003543FFC08E60303FD54C04C2AFAED5457
:100E53003F3BFB0808084300F0D55CCDC21B885814
:100E63007C008C5F8B5E8A5DECC454F0F9EBC45458
:100E73000F49F55978003027027801E55B75F007D3
:100E8300A4F9E5F028F5F0E9A2F013A2F113A2F218
:100E930013F8C3947850027878885B22AA5DAB5E1E
:100EA300AC5F302003020DF6E559C39403400A9466
:100EB300045003020F6C020F33ECC4F9540FFFE923
:100EC30054F0FEEBC4F9540F4EFEE954F0FDEAC4AE
:100ED300540F4DFDC3EA9DFAEB9EFBEC9FFC860588
:100EE30008860608860708084300F08858EF0303BE
:100EF300F9543FFFE954C0CE0303F9543F4EFEE9D2
:100F030054C0CD0303543F4DFDEA2DFAEB3EFBECF9
:100F13003FFC8C5F8B5E8A5DD55C13C21BECC39474
:100F23000C40097C0CE4F55DF55E8C5FC16BC1235D
:100F3300EC0303F9543FFFE954C0FEEB0303F954F8
:100F43003F4EFEE954C0FDEA0303543F4DFDC3EA9F
:100F53009DFAEB9EFBEC9FFC860508860608860738
:100F630008084300F0885880A0ECC423F9541FFFFD
:100F7300E954E0FEEBC423F9541F4EFEE954E0FDAF
:100F8300EAC423541F4DFDC3EA9DFAEB9EFBEC9F7D
:100F9300FC860508860608860708084300F088587B
:100FA300C3EF13FFEE13FEED13FDE10CC3E55D2369
:100FB30023F954FCFAE95403FBE55E2323F954FCBB
:100FC3004BFBE95403FCE55F232354FC4CFCC3E4D3
:100FD3009AFAE49BFBE49CFC24064005E47CFAFAC1
:100FE300FBC2AF8A6C8B6D8C6ED2AF801AE559C38E
:100FF30094024004C22480B4D224C2AF756C4C75F1
:101003006DA0756EFFD2AF3020057F0302102E78DE
:1010130092E6FFC3E55B948240110FC3E55B94A0A6
:1010230040010FC3EF940640027F05E55FC4FC5403
:101033000FFAEC54F0F9E55EC4FC540F49F9EC5493
:10104300F0F8E55DC4540F48F8C3E89440FBE99415
:1010530000FCEA9400FD400CC3EB9401EC9400ED1A
:10106300940050057B01E4FCFD202047C3E49BF87A
:10107300E49CF9E49DFAE8FBE9FCEAFDD3ED13FDFA
:10108300EC13FCEB13FBC2AF8869896A8A6BD2AF9E
:10109300C3EF9403704FC2AF886689678A68D2AF83
:1010A30028F8EC39F9ED3AFAC2AF886389648A65A6
:1010B300D2AF22E4C2AFF569F56A756BECD2AFC269
:1010C300AFF56CF56D756EECD2AFC2AF7563B075ED
:1010D30064FF7565FFD2AFC2AF7566B07567FF7504
:1010E30068FFD2AF2220E111EB28F8EC39F9ED3A91
:1010F300FAC3EF94034016803DE828F8E939F9EA8A
:101103003AFA74FFFBFCFDC3EF94035029C2AF8886
:101113006689678A68D2AFD3E56B13FAE56A13F978
:10112300E569132BFBE93CF9EA3DFAC2AF88638911
:10113300648A65D2AF22C2AF8B668C678D68D2AFEB
:10114300D3E56B13FDE56A13FCE5691328F8EC3965
:10115300F9ED3AFAC2AF886389648A65D2AF223067
:101163002401227A007BFDE5590303543FF99403DC
:101173004005E4FAC399FBD3EB13FBEA13FAD3EB71
:1011830013FBEA13FAC2AF8A558B56D2AF22C2338E
:1011930053A4EFD2845388A5758C0075892A85786A
:1011A3008E7508A785718BC2A9C2BBD2AAD2A8D259
:1011B3008CC22F32FBEA13FA0C802E74FFFBFA80E9
:1011C30026E55FAB5EAA5DC4F8540FFCE854F0CB90
:1011D300C4F8540F4BFBE854F0CAC4540F4AFAEA5C
:1011E30024FFEB34FF50D4E4FCC3EB1370C6EC23B1
:1011F3004B540FC4FBEAC4FA540F4BFBEA54F0FA06
:101203006BC46B540F4A640FFA78B97445C0E07429
:1012130012C0E079757D13EA540F242A83C0E0C01D
:1012230005EAC4540F241F83C0E0C005EB540F2408
:101233001583C0E0C005EBC4540F240A83C0E0C08B
:1012430005227600D23322000C1B24303F4B576615
:10125300727C8693A2AFBC00000000000000000077
:10126300000000000000000000000000000000007B
:10127300000000000000000000000000000000006B
:10128300000000000000000000000000000000005B
:10129300000000000000000000000000000000004B
:1012A300000000000000000000000000000000003B
:1012B300000000000000000000000000000000002B
:1012C300000000000000000000000000000000001B
:1012D300000000000000000000000000000000000B
:1012E30000000000000000000000000000000000FB
:1012F30000000000000000000000000000E7F60806
:10130300A67508A67708797522E7F608A67508A6D4
:101313007608A67508797522E7F608A67708797620
:1013230022E7F608A67708A67508797522E7F60876
:10133300A67508A67508A67608797522E7F608A6A5
:101343007608A67608797522E7F608A67608A675C4
:1013530008797622E7F608A67608A67508A6750822
:10136300797522E7F608A67508A676087976220924
:10137300E7F608A6770879752209E7F608A676083E
:1013830079762209E7F608A67608A6750879752204
:10139300E7F608A67508A67508A6750879762209E2
:1013A300E7F608A67508A6760879752209E7F60810
:1013B300A67508A6750879762209E7F608A67508C2
:1013C300A67508A67508797522901A0D78209132B2
:1013D300E520B4550AA39132E520B4AA028013751F
:1013E30046A57547F1120736910675460075470005
:1013F3008010901A0378807B269132A308DBFA9041
:101403001A2922C2AF91759152901A007403913731
:10141300A374009137A374219137901A0378807BCA
:10142300269136A308DBFA91889166901A2922E463
:1014330093F622E6438F01538FFDFFC3E583941C8C
:10144300400122EF8546B78547B7F0538FFE22430D
:101453008F02438F018546B78547B7901A0DF05326
:101463008FFC22901A0D74559137901A0E74AA911D
:1014730037227A3079807820901A409132E520F330
:1014830009A3DAF7227A307980901A40E391370979
:10149300A3DAF9227C051205CCDCFB22EFC3940707
:1014A300400FEFD3940E5009E570C394065002C366
:1014B30022EF14B40E0040030215599014CC75F0BA
:1014C30003A4C58325F0C583730214F60214F60240
:1014D30014F60214F60214F6021559021503021546
:1014E3001002151D0215280215590215560215334F
:1014F30002153DEF24FEFF7899E6FD12165580563E
:101503007F033032027F017888A60780407F043052
:1015130032027F027888A607802D30323978881608
:1015230016C232803120322E78880606D2328026C7
:101533007888E630E002800F8013901A0BE49364FE
:10154300017888F630E006D230D2318009C230C249
:101553003180031209E6E4F56FF570D322E4F588D0
:10156300780876A7C228F56FF570C2A975892AF5A0
:101573008DF58CC2AFD2AAD2AB757856758E5675DF
:101583008851C2AF7571F175720A7571E275721483
:10159300C2AFD2581208DE7573FE7574FE7575FC02
:1015A3007576F77577F175790AD2AF1205EFE5799C
:1015B300C3940A500122C2AFC2581208DE75790AD9
:1015C300D2AF1205EFE579C3940A5001227571C3B6
:1015D300757228C2AFD2581208DE75731D7574FE7A
:1015E3007575F67576EB7577E075790AD2AF1205E6
:1015F300EFE579C3940A500122C2AFC2581208DE44
:1016030075790AD2AF1205EFE579C3940A50012226
:10161300C3227F087581CD43FF807597DE7597AD33
:1016230075EF06E4F5A9F5A9AE070FA806E4F6EFF2
:1016330070F61207E712087712089A12156050F530
:101643001208ED12090512095D50EA1209FF40F66E
:1016530080E38F088D09C2AF120593E50814601467
:1016630014601814601C1460192404701AAF091252
:1016730006D58013AF091206DB800CAF091206E111
:0C1683008005AF091206E7D2AF0205EFA8
:1019FD00021615030021FFFFFFFFFFFF09FF01FF87
:101A0D0055AA01FFFFFFFFFF03FFFFFF25D0285061
:0D1A1D0004FF02FF7AFF0701FFFF0000FF3A
:101A4000234A5F4C5F313523202020202020202096
:101A500023424C48454C492445464D3842313023B9
:101A60002020202020202020202020202020202076
:101C0000C2AFC2D37597DE7597AD7581C075A90057
:101C100075A90043FF80752438752503B1DE752949
:101C2000A5752AF143F11053A4EFD28475D4FF7542
:101C3000E3407DFA780379E67C1075220075230075
:101C4000901DEB7B06752498752501308402814B2D
:101C5000208408D8FBD9F9DCF781BD308408D8FB93
:101C6000D9F9DCF781BDB19EE493A3C39A6004DD8A
:101C7000C381BDDBDBB190600281347B08E493FA61
:101C8000A3B171DBF87A30B171752200752300B110
:101C900090EAFCEBFDC3ED94FE400EB1908A278BD9
:101CA00028ED30E0048A828B83B1907AC270D8C369
:101CB000ED94FE601950CEBD0029EC600F75200038
:101CC0007521FF752900752A000200008100A827F0
:101CD000A9280809D804D90281E0B194EAF281D494
:101CE0000D81A9C3ED94035051EDA2E092007AC595
:101CF000C3E5829400E583941C508C200010438F30
:101D000002438F018529B7852AB7F0300027A8271D
:101D1000A9280809438F01538FFDD804D902A135A2
:101D2000C3E583941C4003A3A11AE28529B7852A41
:101D3000B7F0A3A11A538FFC81857AC1BD030CE4CF
:101D400093A3FAB155DCF8B14D81858187AA22AB06
:101D500023B171EBFAEA6222752608C3E52313F575
:101D600023E52213F52250066323A0632201D52622
:101D7000EAB1DEB1DE75260AEAF4200102D284302F
:101D80000102C284B1DEC3134002C201D526EB2298
:101D9000B194EAFB208402A194308402A1997526B3
:101DA00008AE24AF25C3EF13FFEE13FEB1E2B1DEA0
:101DB000C3EA133084024480FA30E703632201C38C
:101DC000E52313F523E52213F52250066323A063D0
:101DD0002201D526D9E52265236523F52222AE24EA
:101DE000AF250E0FDEFEDFFCD20122424C48656CAF
:091DF0006934373164E8B10601E1
:00000001FF
